:100000000C945B020C9478020C9478020C947802A5
:100010000C94C52A0C9478020C9478020C94780203
:100020000C9478020C9478020C9450250C940C25B6
:100030000C944C260C9478020C9478020C94780260
:100040000C9478020C9478020C9478020C94780248
:100050000C9478020C9428260C9478020C94780264
:100060000C9478020C9478020C9478020C94780228
:100070000C9478020C9478020C9478020C94780218
:100080000C9478020C9478020C9478020C94780208
:100090000C9478020C9478020C9478020C947802F8
:1000A0000C9478020C9478020C94780229003500A4
:1000B00014001A000800150017004B00E0000400AF
:1000C0001600070009000A000000E2001D001B00E6
:1000D00006001900050000000000000000004C426E
:1000E0002A22E34130002F00130012000C001800F8
:1000F0001C004E00343133000F000E000D000B00C9
:1001000000003134380037003600100011000000C4
:100110000000000000002B422C32284101002D027B
:100120003A003B003C003D003E00010057001E022B
:100130001F02200221022202000067001E001F0091
:10014000200021002200000000000000000001004B
:10015000010001004500440043004200410040000E
:100160003F00010056002702260225022402230236
:1001700000000100270026002500240023000000C5
:10018000000000000000010001000100A800530071
:1001900054005F00600061005600A9006700550030
:1001A0005C005D005E005700000001006200590025
:1001B0005A005B0085000000000000000000010004
:1001C000010001004D0039004700480046004A0088
:1001D0000100AA00650049004F00520050000100D4
:1001E000000001000100010051004D00010000006D
:1001F00000000000000001000100010001000100FA
:1002000001000100010001000100010020782378B5
:10021000257827782978010000002178247826782D
:1002200028782A780100000000000000000001008A
:1002300001000100010001000100D200DE00D10038
:10024000D900010001000100D000CD00CF00DA008C
:10025000000001000100DF00CE00DD000100000011
:100260000000000000000100010001000001010188
:100270000101010101010202020202020202020363
:100280000303030303030304040404040404050533
:1002900005050506060606060707070707080808F6
:1002A00008090909090A0A0A0B0B0B0C0C0C0D0DA5
:1002B0000D0E0E0E0F0F0F1010111111121213133D
:1002C0001414151516161717181819191A1A1B1BB6
:1002D0001C1D1D1E1E1F2020212222232424252612
:1002E00026272829292A2B2C2D2D2E2F303132324A
:1002F000333435363738393A3B3C3D3E3F40414256
:10030000434445464748494A4C4D4E4F505153543B
:10031000555658595A5B5D5E5F61626465666869EF
:100320006B6C6D6F7072737577787A7B7D7E80826F
:10033000838587888A8C8E8F91939596989A9C9EB8
:10034000A0A2A3A5A7A9ABADAFB1B3B5B7BABCBEC8
:10035000C0C2C4C6C9CBCDCFD1D4D6D8DBDDDFE295
:10036000E4E7E9EBEEF0F3F5F8FAFDFF0501090229
:10037000A10185020901A10005091901290815003B
:1003800025019508750181020501093009311581A2
:10039000257F95027508810609381581257F95010D
:1003A00075088106050C0A38021581257F950175AF
:1003B000088106C0C005010980A101850319012A31
:1003C000B700150126B700950175108100C0050C16
:1003D0000901A101850419012AA002150126A00224
:1003E000950175108100C005010906A101050719D5
:1003F000E029E71500250195087501810295017531
:100400000881010507190029FF150026FF00950640
:1004100075088100050819012905150025019505B4
:1004200075019102950175039101C009023B00021B
:100430000100A0FA090400000103010100092111D3
:10044000010001224400070581030800010904019D
:10045000000103000000092111010001227B0007B7
:100460000582032000011201000200000008EDFED9
:100470000000010001020001160341006E00670048
:1004800065006C00570069006E0067007300000093
:10049000200344006F007200790061006E002000AC
:1004A00061006E00640020004E004D0031003700F6
:1004B00000000403090411241FBECFEFDAE0DEBF01
:1004C000CDBF25E0AEE7B2E001C01D92AF36B20766
:1004D000E1F712E0A0E0B1E0E2E0FCE502C0059047
:1004E0000D92AE37B107D9F70E9473260C948A2D6E
:1004F0000C94000090916705937061F081110BC01E
:100500009460909367051092370180916605816031
:10051000809366050895813210F09068F2CF880FBD
:10052000880F982BEECF982FE0915E05409125051E
:1005300057E0E41302C080E008952E2F30E05E9F64
:10054000F0011124EA5DFA4F8181681306C08081B1
:10055000981303C085818111EFCFF9013196E770BF
:10056000E8CFFC01AC014C5F5F4F8FEF91E321912D
:10057000822728E030E087FF09C0880F89272150B3
:100580003109C9F7E417F50791F70895880FF7CFF8
:1005900090916705937071F0809368056093690589
:1005A000433808F042E840936A058091660581600F
:1005B000809366050895E8EDF0E080818E7F80836A
:1005C0001092E2001092DA001092E100A0EEB0E08A
:1005D0008C9181608C9380818F77808319BCA7ED8B
:1005E000B0E08C918E7F8C9380818F7E808310927F
:1005F0000E0508952091E4003091E50095E6A901EB
:100600002091EC00822F817020FF06C08091E800CD
:1006100080FF06C080E008952091E80022FD1AC006
:1006200080911B05882389F0853089F08091EB004B
:1006300085FD0FC02091E4003091E500421753077B
:10064000F9F29150E1F684E0089582E0089583E0A4
:10065000089581E0089580911D0587FF13C0809162
:10066000E80082FF06C08091E8008B778093E80065
:1006700004C080911B058111F2CF089580911B0564
:100680008823D9F38091E80080FFF8CF8091E800BB
:100690008E77ECCF982F9093E900242F762F50E09F
:1006A000891731F07091EC002091ED005091F0002D
:1006B00021FD07C09F5F973071F78093E90081E0CB
:1006C00008953091EB003E7F3093EB003091ED00C8
:1006D0003D7F3093ED003091EB0031603093EB00C3
:1006E0007093EC002093ED005093F0002091EE0009
:1006F00027FDE0CF80E00895B0E0A0E0E2E8F3E07D
:100700000C94EC2BC8EDD0E088818F7E8883E7EDD8
:10071000F0E080818160808384E082BF81E080930B
:100720000E0588818E7F888302EE10E0F80110822A
:100730001092DA0081EEC82ED12CF6011082888149
:100740008F77888388818068888388818F7D88837C
:1007500019BC10921B0510921C0510921A051092DC
:10076000190590EEE92EF12CF70180818B7F8083B3
:1007700088818160888342E060E080E00E944A03D3
:10078000F60180818E7F8083F80180818160808383
:10079000808188608083F70180818E7F808388815B
:1007A00080618883CDB7DEB7E8E00C94082CFC01AB
:1007B000CB0120912305309124052617370790F0AF
:1007C000009729F42091E8002E772093E80040E07C
:1007D000009751F4411108C08091E80082FF31C0B8
:1007E00080E00895C901F3CF20911B052223A9F1D0
:1007F0002530A9F12091E80023FD2DC02091E800CB
:1008000022FDEACF2091E80020FFE2CF3091F300F3
:100810002091F200009719F02830310558F041E09E
:100820002830310509F040E02091E8002E77209330
:10083000E800CECF41914093F10001972F5F3F4FE9
:10084000E9CF80911B05882341F0853041F08091EC
:10085000E80083FFC1CF81E0089582E0089583E03E
:10086000089508958091100508959C014FB7F8945C
:1008700080910A0590910B05A0910C05B0910D0592
:100880004FBF821B930B0895A4E0B0E0EAE4F4E0CC
:100890000C94F22B8FB7F89420910A0530910B0538
:1008A00040910C0550910D0529833A834B835C835D
:1008B0008FBF69817A818B819C812496E2E00C94C0
:1008C0000E2C2FB7F89480910A0590910B05A091FA
:1008D0000C05B0910D052FBF08959C01FC013296C7
:1008E0008FEF90E04191461751F08F3F19F441117D
:1008F00001C0892F9F5F9630A9F78F3F09F40895B3
:10090000280F311D87FD3A95F90162830895A3E010
:10091000B0E0EDE8F4E00C94F22B9C018091070527
:100920009091080582179307A1F030930805209352
:100930000705E0910505F0910605309751F084E038
:1009400089833B832A830084F185E02DCE010196C3
:1009500009952396E2E00C940E2CA3E0B0E0E3EBC3
:10096000F4E00C94F22B9C01809103059091040516
:1009700082179307A1F03093040520930305E091BB
:100980000505F0910605309751F083E089833B839C
:100990002A830084F185E02DCE01019609952396E6
:1009A000E2E00C940E2C80910105882359F0E0912F
:1009B0000505F0910605309729F00190F081E02DB2
:1009C0000995089580E008950E9461042091FD0436
:1009D0003091FE04232B21F08093F9049093FA04C4
:1009E0002091FF0430910005232B21F08093F70420
:1009F0009093F804E0910505F0910605309749F0D1
:100A000082E08093FB040680F781E02D8BEF94E079
:100A1000099508958091F60480FD16C081FD16C0E9
:100A200082FD16C08091F5048823A1F0883280F4FD
:100A300028E0829FC001112468E270E00E942D2C02
:100A4000862F672B39F0089582E0089584E0089599
:100A500088E0089581E008958091F60480FD14C037
:100A600081FD14C082FD16C08091F404882381F0BA
:100A70008E3180F420E5829FC00111246EE170E088
:100A80000E942D2C862F089584E1089588E2089510
:100A900088E0089580E50895282F35EB2303C001F1
:100AA000112497FF04C080589109892F0895805818
:100AB0009F4FFBCFFA01882311F009950895FB01A0
:100AC000FCCFFC0180910205811123C0E731F105C3
:100AD0001CF17797CF01880F991FDC01AE0FBF1F64
:100AE000AC5CBB4F11963C911197361307C03C91FB
:100AF000341304C012963C91321771F031E03093F8
:100B00003304E80FF91FEC5CFB4F618340832283C1
:100B100003C0E731F105F4F208951092330408950B
:100B2000E7E6F5E024813AE0231B08F420E0248383
:100B3000809166058160809366050895E7E6F5E09B
:100B400024813AE0230F08F42FEF24838091660577
:100B50008160809366050895E7E6F5E0438128E02B
:100B6000421B08F440E08181628190E00E94C8024B
:100B70000895E7E6F5E0438128E0420F08F44FEFDF
:100B80008181628190E00E94C8020895E7E6F5E065
:100B9000628128E0621B08F460E08181438190E07B
:100BA0000E94C8020895E7E6F5E0628128E0620F3E
:100BB00008F46FEF8181438190E00E94C80208959C
:100BC000E7E6F5E08181438162818850990B0E94BC
:100BD000C8020895E7E6F5E0818190E043816281F3
:100BE00008960E94C802089590916705969596957B
:100BF0008FEF890F913009F480E20E947A02089504
:100C000080916705869586958F5F813208F081E037
:100C10000E947A0208959DE0899F802D1124980FEB
:100C2000913408F090E420910205222321F09831BC
:100C300028F097E10895873108F487E10895E42FBB
:100C4000F0E0EE0FFF1FE254FE4F9081921B97FDE4
:100C50009195292F38E1239F212D1124620F0895AA
:100C60000F931F93522F10E0F801EE0FFF1FE25475
:100C7000FE4F9081905797FD9195000F111FF8013D
:100C8000EA57FE4F01AD0052110B50039001519FE6
:100C9000300D112408E310E0091B110997FD13958D
:100CA0004003F001419FF00D1124E20FF31F9F015B
:100CB000220F331F2E0F3F1F37FF02C021583F4F17
:100CC000220F232F221F330B620F1F910F910895C4
:100CD0000F931F93522F10E0F801EE0FFF1FEA57FA
:100CE000FE4FA1ADA052BB0B9D015203F001539FDB
:100CF000F00D1124000F111FD801A254BE4F0C910A
:100D00000057110B40039001419F300D11242E0F0D
:100D10003F1F37FF02C0215C3F4F96E03595279576
:100D20009A95E1F7620F1F910F9108950F931F930A
:100D3000522F10E0F801EE0FFF1FEA57FE4FA1AD52
:100D4000A052BB0B9D015203F001539FF00D1124E3
:100D5000000F111FD801A254BE4F0C910057110B68
:100D600040039001419F300D11242E0F3F1F37FF8C
:100D700002C021583F4F220F232F221F330B620F37
:100D80001F910F910895EF920F93972F23E0029FE9
:100D9000B0011124759567956E0D792F0F91EF9025
:100DA0000895322F50E0FA01EE0FFF1FEA57FE4F71
:100DB00091AD905297FD9195440F551FFA01E25461
:100DC000FE4F2081231B330B290F311D97FD3A95D0
:100DD000620F0895E42FF0E0EE0FFF1FEA57FE4F79
:100DE00061AD621B0895E42FF0E0EE0FFF1FE254A7
:100DF000FE4F6081621B0895622F0895582FA22F25
:100E0000E42FF0E0EE0FFF1FE254FE4F208134EE9E
:100E1000239F212D112490E030E0245E3F4F2A1BB8
:100E2000310937FF03C031952195310943E0220F85
:100E3000331F4A95E1F7821B930B97FD80E0282F23
:100E4000259F212D1124822F08951F93172F922F54
:100E5000E42FF0E0EE0FFF1FE254FE4F208134EE4E
:100E6000239F212D1124472F50E030E0245E3F4F77
:100E7000291B310937FF03C031952195310993E0D2
:100E8000220F331F9A95E1F7421B530B57FD40E0A9
:100E9000742F719F712D11241F9108950E94610577
:100EA0000895FF920F931F93CF93DF93182F062F70
:100EB000F42ED0E0C0E02F2D402F612FCE010E94F4
:100EC0004E072196C034D105B1F7CDB7DEB7E5E0C6
:100ED0000C940B2CFC019B01009729F480E077FF18
:100EE0002BC080E80895AC0197FF04C04427552724
:100EF000481B590BB901640F751F37FD10C0241B27
:100F0000350BC901A5E0880F991FAA95E1F70E944A
:100F10002D2C80E2861BF7FF0FC081950895CB0131
:100F200065E0880F991F6A95E1F7BA01621B730BA0
:100F30000E942D2C80E6EECF0895EF920F93CF9371
:100F4000DF93D72FC82FBA01C9010E190E946A0773
:100F5000602F681B7D2F8C2FDF91CF910F91EF9029
:100F600008950F93CF93DF93D72FC82FBA01C901EC
:100F70000E946A07682F600F7D2F8C2FDF91CF9121
:100F80000F910895EF920F931F93CF93DF93D62F76
:100F9000C72F182FBA01C9010E19010F0E946A0745
:100FA000081B019F012D11246D2F7C2F802FDF91B5
:100FB000CF911F910F91EF900895EF920F931F9390
:100FC000CF93DF93D62F172FC82FBA01C9010E195F
:100FD000010F0E946A07702F781B719F712D1124D9
:100FE0006D2F8C2FDF91CF911F910F91EF9008956E
:100FF0000F931F93CF93DF93D62FC72F182FBA01CC
:10100000C901212F201B022F0E946A07982F990FD8
:10101000990F282F291B200F219F212D11246D2F7F
:101020007C2F822FDF91CF911F910F9108950F9305
:101030001F93CF93DF93D62F172FC82FBA01C90163
:10104000212F201B022F0E946A07982F990F990FBA
:10105000782F791B700F719F712D11246D2F8C2F9C
:10106000DF91CF911F910F910895982FE82F96FD52
:10107000E0952E2F2F7096FD2F5FE695E695E6956D
:10108000E670F0E0E258FE4F8181829F802D212D95
:10109000112482958F702295207F822B2081820FD0
:1010A00097FD8195805808950F931F93CF93DF93F9
:1010B0008B01D82FC42F822F0E943508EC2FF0E02F
:1010C000EE0FFF1FE254FE4F90819058980F97FD4E
:1010D0009195990F692F2CE0629F612D1124600F6B
:1010E000712F8D2FDF91CF911F910F910895409116
:1010F0002F015091300125E038E0429FC001439F0D
:10110000900D529F900D1124875E994C9093300161
:1011100080932F01890F08959C018230910508F476
:1011200008959FEF213E8EE1380740F4C90145E064
:10113000969587954A95E1F798E0980F61E0E62F3C
:10114000E90FFF27FF1FAF0155954795842F449F57
:10115000F001459FF00DF00D11242E173F0738F4D4
:101160009FEF940F961758F78FEF860F08954F3F14
:10117000E9F361E0640FF6CF0F93CF93DF93D72F9E
:10118000C82FF90147FD419528E330E0241B3109C0
:1011900047FD3395229FA001239F500D500D112430
:1011A000EE9FC001EF9F900D900D1124840F951FAD
:1011B0000E948C08982F990F692F680F600F7D2F60
:1011C0008C2FDF91CF910F9108959C0190E080E0EA
:1011D000269F812D369F800D911D11240895A4E036
:1011E000B0E0E5EFF8E00C94F22B20916B0530E1D4
:1011F000230F08F42FEF60E1822F90E00E94E508B2
:10120000BC0188EB9BE00E94192CB0E0A0E0CD016E
:101210002496E2E00C940E2C982F809102058823EE
:1012200029F081E0973128F080E003C081E090341C
:10123000D8F70895B0E0A0E0E0E2F9E00C94EA2BE2
:10124000262F472FE82FF0E0E459FD4F711109C018
:101250006491862FE62F7E2FCDB7DEB7EAE00C949F
:10126000062CE72EF12CE49186E0689F8001112482
:10127000CFEFD0E0C801BE010E94192CDB0130E0A5
:10128000220F331F55E5569FC001579F900D112423
:10129000281B390B622F660F260FCE018E199F096E
:1012A000E89F6001E99FD00C11246D2D429FA001A1
:1012B0001124452F5527CE01841B950BE89FA001D3
:1012C000E99F500D1124852F5E01A21AB108AE9C32
:1012D0009001AF9C300DBE9C300D1124232F33277D
:1012E000C21BD30BEC9F9001ED9F300D1124A33056
:1012F000B105B1F00C3F93E0190760F4A130B105DE
:1013000099F01297A9F00F3F110508F0A4CF8D2D89
:10131000632FA1CFA430B10571F01697C1F39BCF15
:10132000652F8E2FED2D97CF6E2FE52F8D2D93CF1F
:10133000832F6E2FF7CF8E2FE32F8DCFB0E0A0E05D
:10134000E4EAF9E00C94ED2BEC01FC01E25CFD4FCA
:101350008081682349F1D090690500916A05109158
:101360006805E12EF12C0E947708282FC7018C54C4
:101370009F4F68E671E00E942D2C8E199F0997FD02
:10138000039695958795959587952370612F289F4E
:10139000600D11247D2D802F0E941A09462F672F82
:1013A000282FCE010E944E07CDB7DEB7E7E00C94A0
:1013B000092CEF92FF920F931F93CF93DF937C0141
:1013C000809134010E940B06C82F192F60916B0584
:1013D0006695669521E0620F08F46FEF80915F05D6
:1013E000909160050E94E508082FD0E0C11740F0F9
:1013F000812F0E940C09CDB7DEB7E6E00C940A2CD1
:10140000FE01E25CFD4F808190913501892391F0CE
:10141000609168057091690580916A05202F4C2FB5
:10142000F70109950E941A09462F672F282FCE0130
:101430000E944E072196DACFA4E0B0E0E2E2FAE0A3
:101440000C94EC2B6C01809134010E940B068B8371
:10145000F92E60916B056695669580915F05909178
:1014600060050E94E508182F80E4810F0E9435086E
:1014700080588983812F0E94350880588A839B81F8
:10148000892F90E09C838B839B819F1538F08F2D53
:101490000E940C092496E8E00C94082CEB81FC8156
:1014A000E25CFD4F8081909135018923A9F0609124
:1014B00068057091690580916A05E12E0B812A818A
:1014C0004981F60109950E941A09462F672F282F96
:1014D0008B819C810E944E078B819C810196D2CF8B
:1014E000B0E0A0E0E6E7FAE00C94E62B3C01809146
:1014F00034010E940B06C82F192F60916B05669569
:1015000080915F05909160050E94E508F82ED0E07B
:10151000CE01880F991F9C012A573E4F6901C117C0
:1015200040F0812F0E940C09CDB7DEB7EEE00C949D
:10153000022CFE01E25CFD4F8081909135018923F0
:1015400079F1F60180AD282F2057330B590181AD79
:10155000E82FE052FF0B4F01AA9C9001AB9C300D8D
:10156000300D1124EE9FC001EF9F900D900D1124BE
:10157000820F931F0E948C08082F6091680570915C
:10158000690580916A05EF2C9401A501F301099585
:101590000E941A09462F672F282FCE010E944E075E
:1015A000F2E0CF0ED11C2196BACFAF92BF92DF925C
:1015B000EF92FF920F931F93CF93DF935C01809183
:1015C00034010E940B06C82F192F60916B05669598
:1015D00080915F05909160050E94E508D82ED0E0CB
:1015E000CE01880F991F9C012A573E4F7901C117E0
:1015F00068F0812F0E940C09DF91CF911F910F910C
:10160000FF90EF90DF90BF90AF900895FE01E25CF5
:10161000FD4F8081909135018923C1F0F70121AD03
:101620002052330B40AD4057550B609168057091C7
:10163000690580916A050D2DF50109950E941A0929
:10164000462F672F282FCE010E944E07F2E0EF0EA3
:10165000F11C2196CCCF1F93CF93DF93EC01FC01BB
:10166000E25CFD4F80816823B1F00E947708182F5B
:101670000E94770820E8829FC00111247FE7790F3C
:10168000612F80916A050E941A09462F672F282F23
:10169000CE010E944E07DF91CF911F91089580E007
:1016A0000895F894E82FE295EF70F0E041A18F7073
:1016B00021E030E0B90102C0660F771F8A95E2F79A
:1016C000CB01962F9095942391A392A1892B82A36D
:1016D00078940895A4E0B0E0E0E7FBE00C94F22BEE
:1016E00080910105882371F00E94440469837A8304
:1016F0008B839C8369817A818B819C812496E2E033
:101700000C940E2C0E94440469837A838B839C83FF
:101710008091E8029091E902A091EA02B091EB0277
:1017200029813A814B815C81280F391F4A1F5B1F39
:1017300029833A834B835C83DDCF9091FA0292FF39
:1017400010C041E0282F2471243009F040E031E03E
:10175000282F2871283009F030E0431711F02CE0D1
:10176000822793FF10C041E0282F2471243109F013
:1017700040E031E0282F2871283109F030E043178C
:1017800011F02CE082273091FB0230FF10C051E0B5
:10179000282F2171213009F050E041E0282F2871D5
:1017A000283009F040E0541711F029E0822731FF7A
:1017B00010C041E0282F2171213109F040E031E0D3
:1017C000282F2871283109F030E0431711F029E063
:1017D000822794FD877E0895803E9105C1F1C8F46B
:1017E0008133910509F47DC048F48932910509F4EB
:1017F0006DC08A32910509F47BC008958933910543
:10180000D1F082389105B9F08533910509F459C0BA
:101810000895843E9105C1F138F4823E910521F18D
:10182000833E910531F10895863E9105C1F1873ED1
:101830009105E1F108952091FA02237009F065C045
:101840002091FB0223FF14C089E290E008952091CB
:10185000FA0220FD43C03091FB0230FF09C024FF93
:101860004EC090E080E008952091FA0222FDF7CF6B
:1018700008952091FA0222FD45C03091FB0230FD0F
:1018800044C024FFF5CFEDCF2091FB0221FFF0CF24
:101890008091FA0284FDE5CF87EE90E008952091D3
:1018A000FA0223FFE5CF24FDDCCFF6CF2091FA0228
:1018B00023FD2EC03091FB0231FFE3CF84EE90E098
:1018C00008952091FA0225FFD3CFBECF2091FA02CE
:1018D00025FD21C02091FB0223FFCACF89E390E0C0
:1018E000C7CF2091FA0226FFC3CF8AE290E0089585
:1018F0002091FA0226FFBCCF81E390E0089583EEA9
:1019000090E0089582EE90E0089580EE90E00895D2
:1019100086EE90E0089585E390E008957830B8F47D
:101920006730A8F48430B0F4E62FF0E097E0799FB8
:10193000E00DF11D112498E3899FE00DF11D1124A4
:10194000EE0FFF1FE455FF4F85919491089580E0BD
:1019500090E0089581E0FCCF1F93CF93DF930E9426
:10196000EC0BEC018115924508F05FC0C11580E5D4
:10197000D80708F0DDC0C03ED10538F5CD3CD10513
:1019800008F0AEC0C83AD10580F4C53AD10508F0D8
:10199000A4C0C130D10509F443C0CE010497813AF7
:1019A0009105F0F1D0E0C0E03BC0CE01885A91092A
:1019B0004B97C0F7C85AD0E0CC0FDD1FC55CDE4F97
:1019C0000990D881C02DD4642BC0C11590E4D907EB
:1019D000F0F4C11520E2D20708F0C4C0C83ED1051A
:1019E000F8F0CE019A9581159F41E0F68D2F0E9467
:1019F0009D0B182FCE0199270E94EC0BC12FD0E030
:101A0000DC2FCC27CC27DF71C82BD92B09C0CE0106
:101A100099270E94EC0BCC27DF70C82BD92BD06AFA
:101A2000CE01DF91CF911F910895C03882E5D8078C
:101A3000B8F5C03692E5D90708F05BC0C03422E59E
:101A4000D207C8F4C03282E5D80708F04BC02C2F6B
:101A50002695269590E2299F900111248C2F837062
:101A6000C1E0D0E002C0CC0FDD1F8A95E2F7C22BA7
:101A7000D32BDD68D5CF2C2F26952695277080E2B5
:101A8000289F900111248C2F8370C1E0D0E002C008
:101A9000CC0FDD1F8A95E2F7C22BD32BDC68C0CFB9
:101AA000C03C92E5D90760F48C2F8F71C03AD245C3
:101AB000A8F5C82FD0E0DC2FCC27C46FD06AB0CFF8
:101AC000CE01805C9245809708F06CCFDC2FCC274C
:101AD000CC27DF71C06FD06AA3CFA497D064A0CF0A
:101AE000D0659ECFCF71D0E0DC2FCC27C16FD06AFC
:101AF00097CF2C2F26952695277080E2289F90015E
:101B000011248C2F8370C1E0D0E002C0CC0FDD1F08
:101B10008A95E2F7C22BD32BDA6882CF0E949D0B05
:101B2000C82FD0E0DC2FCC27CC27DF71D06278CF54
:101B30008C2F8F710E949D0B55E0D695C7955A95B5
:101B4000E1F7CF70D0E0DC2FCC27282F30E084FFE6
:101B500005C044E0220F331F4A95E1F7C22BD32B77
:101B6000D0695ECF8D2F8F710E949D0B182FCE01F3
:101B700099270E94EC0BC12FD0E0DC2FCC27CC277B
:101B8000DF71C82BD92BD2CF982F90958091B802B6
:101B900089238093B802089580915E059091250570
:101BA000981301C008958F5F8770FACFB0E0A0E06E
:101BB000ECEDFDE00C94EB2B8C01E090F802F09042
:101BC000F9028091F6029091F702E82AF92ACFE013
:101BD000D0E0CC24C394D12CBC2EC6010C2E02C064
:101BE000880F991F0A94E2F78E219F21892B49F4CF
:101BF000219790F7B12C8B2DCDB7DEB7E9E00C948F
:101C0000072CB8018C2F0E948E0C0E94AC0C0197FF
:101C100079F3F1CFCF93DF93D82FC92F0E94D60D40
:101C20006D2F7C2F0E948E0C0E94AC0CDF91CF9107
:101C30000895983078F5873068F5E82FF0E087E070
:101C4000989FE00DF11D11249E2F977083E0F6956B
:101C5000E7958A95E1F7EE0FFF1FEE0FFF1FE6579E
:101C6000FD4F50E040E080E0219130E0092E02C0BD
:101C7000369527950A94E2F721703327042E01C088
:101C8000220F0A94EAF7822B4F5F5F4F44305105D1
:101C900059F7089580E00895983098F5873088F5D1
:101CA000E82FF0E087E0989FE00DF11D11248E2FC2
:101CB000877041E001C0440F8A95EAF783E0F6950A
:101CC000E7958A95E1F7EE0FFF1FEE0FFF1FE6572E
:101CD000FD4F30E020E070E05191DF011197CB0122
:101CE000022E02C0969587950A94E2F7817081953D
:101CF0008527842385278C932F5F3F4F2430310520
:101D000059F708959C0186709927069731F4286049
:101D10003093F9022093F8020895277FF9CF21E04C
:101D200030E002C0220F331F8A95E2F720953095EC
:101D30008091F8029091F902822393230E94820EEF
:101D400008959091AD02809589238093AD02282F4C
:101D5000277069F4891759F09091FB0292FF07C030
:101D60008695869586950E948F0E1092AD020895F5
:101D700021E030E002C0220F331F8A95E2F7809104
:101D8000F8029091F902822B932B0E94820E089503
:101D90009093F7028093F6020895FC0184818823D2
:101DA000A1F0808191810E940A0E282F92959F7048
:101DB000963091F060F4925F9F70923030F481E041
:101DC000203F81F030F4283E30F080E004C09A5F7C
:101DD000F3CF243FD1F7089581E0283E20F0213F42
:101DE000A1F7F9CF089508954091FD049091FF0463
:101DF00020910005662309F469C0942B922B209151
:101E0000FE04922B31F098E09093F40491E09093CB
:101E1000F5048D3C41F40E942C0581958093FE04CD
:101E20000E94E40408958E3C19F40E942C05F6CF1C
:101E30008F3C31F40E942C0581958093FD04F0CFF6
:101E4000803D19F40E942C05F8CF893D29F40E94A9
:101E50000A058093FF04E4CF8A3D21F40E940A051D
:101E60008195F7CF8B3D31F40E940A0581958093CF
:101E70000005D6CF8C3D19F40E940A05F8CF9FE2E9
:101E8000980F983070F4815D990B21E030E001C02B
:101E9000220F8A95EAF78091FC04822B8093FC0440
:101EA000BFCF8D3D31F48091F60481608093F604BC
:101EB000B7CF8E3D21F48091F6048260F7CF8F3D3D
:101EC00009F0AECF8091F6048460F0CF8D3C59F4D8
:101ED0008091FE0487FF0DC01092FE0441110BC0DB
:101EE0001092F40408C08E3C81F48091FE04181610
:101EF0009CF3442381F08091FF0490910005892B8D
:101F000009F08ECF1092F5048BCF8F3C49F447FF38
:101F1000F0CF1092FD048091FE048111ECCFE0CF50
:101F2000803D19F41416ACF3E4CF893D29F4191659
:101F300004F71092FF04DDCF8A3D19F497FFD9CF43
:101F4000F8CF8B3D29F427FFD4CF10920005D1CFD5
:101F50008C3D19F41216CCF3CCCF9FE2980F983039
:101F600090F4815D990B21E030E0B90102C0660F69
:101F7000771F8A95E2F7CB0180959091FC04892325
:101F80008093FC04B6CF8D3D31F48091F6048E7FB2
:101F90008093F604AECF8E3D21F48091F6048D7FC0
:101FA000F7CF8F3D09F0A5CF8091F6048B7FF0CF5E
:101FB000A6E0B0E0EEEDFFE00C94F12B49835A83EC
:101FC000392F89819A81332399F0222389F00E9445
:101FD000D60D182F682F89819A810E944C0E698135
:101FE0007A81812F0E948E0C2696E3E00C940D2CB2
:101FF0000E94190E182FF3CF0F931F93CF93DF93E7
:102000008B01EA0190911B05943061F58093E90002
:102010008FEF9091E800815095FD06C095ED9A955F
:10202000F1F700008111F5CF8091E80085FF1AC01B
:102030000E94FA02811111C08091E80085FD06C05E
:102040008091E8008E778093E800F2CFF8018191CB
:102050008F018093F100219779F78091E8008E77C6
:102060008093E800DF91CF911F910F910895BC01FB
:1020700043E050E082E00E94FC0F0895BC0146E07E
:1020800050E082E00E94FC0F0895CF93DF93D82F99
:10209000C92F48E050E0682F792F81E00E94FC0FA3
:1020A00088E0ED2FFC2FA1E1B5E001900D928A951B
:1020B000E1F7DF91CF91089580913304882341F1B6
:1020C000529A3BB13B7F2BB124604FB7F89484E325
:1020D00094E0FC010196508168E02BB9000000C03B
:1020E00057FF3BB9550F000000C000C000C03BB90E
:1020F00000C06A9591F754E0843F950751F74FBFB0
:102100008FE594E00197F1F700C0000010923304CE
:102110000895B0E0A0E0EFE8F0E10C94EA2BF82E8F
:10212000E92ED62EC72E8A018091E702AA24A39415
:10213000B12C8A3018F48AE0A82EB12CC1E0D0E08E
:102140006D2D7C2D8F2D9E2DF8010995811104C0D8
:102150002196AC16BD062CF4CDB7DEB7EAE00C94A0
:10216000062CCC9F9001CD9F300D300D112490E0B6
:1021700080E045E34A95F1F7000001968217930746
:10218000C1F7DECFA6E0B0E0E8ECF0E10C94E52B7F
:102190000E946A0B60930E0370930F0380931003E9
:1021A0009093110320916705322F33703D833323C1
:1021B00021F0422F469546954D83309137013230BC
:1021C00009F4F8C580F4311115C010923401609300
:1021D0005F0570936005809361059093620581E0CF
:1021E0008093370103C0333009F4EEC52696EFE043
:1021F0000C94012C809132015D81581322C0237010
:102200004091310150E081E02417150609F480E087
:1022100081708093360180916C05909135019817FB
:1022200039F08093350140E060E080E00E94510782
:102230006D81613260F4E62FF0E0E457F24D0C94CA
:10224000412C81E0E5CF80913601811102C080E010
:1022500031C140E060E080E00E945107F8CF8091FA
:1022600034010E940B06082F9983609168057091D4
:10227000690580916A050E941A09F62EE72ED82E6C
:1022800010E07981071720F0872F0E940C0912C1F6
:10229000F801E25CFD4F808190913501892331F096
:1022A0002D2D4F2D6E2DC8010E944E070F5F1F4F21
:1022B000E8CF809134010E940B06082FD92EF090B0
:1022C000690510916A05809168058983682F7F2DC3
:1022D000812F0E941A09C62EB72EA82E60916B0579
:1022E0009981690F7F2D812F0E941A096983F72E2A
:1022F000E82E10E00D1510F08D2DC7CFF801E25C2F
:10230000FD4F808120913501282359F02E2D4981E0
:102310006F2D80FD03C02A2D4C2D6B2DC8010E940E
:102320004E070F5F1F4FE6CF809134010E940B06CE
:102330009983E0906905D0906A0520916B0530E49F
:10234000F32E3F2D329F312D1124F32E082F10E054
:102350004981041710F0842F98CFF801E25CFD4FFB
:102360008081909135018923B9F0F801EE0FFF1FAC
:10237000EA57FE4F81AD82958F70609168058F9D01
:10238000600D11247E2D8D2D0E941A09462F672F76
:10239000282FC8010E944E070F5F1F4FD9CF809191
:1023A00034010E940B069983E0906905D0906A057C
:1023B00020916B0590E4F92E5F2D529F512D112431
:1023C000F52E082F10E06981061710F0862F5DCFDB
:1023D000F801E25CFD4F8081909135018923D9F0AD
:1023E000F801EE0FFF1FEA57FE4F60ADF69EB001F9
:1023F000112485E0759567958A95E1F780916805C8
:10240000680F7E2D8D2D0E941A09462F672F282FC9
:10241000C8010E944E070F5F1F4FD5CF8091340136
:102420000E940B06082F9983F090680510916905AA
:10243000E0906A0560916B0566956695669580915A
:102440005F05909160050E94E5080E94350820E82C
:10245000280F27FD2195220F7E2D279F212D112446
:102460006F2D712F822F0E941A09F62EE72ED82E7B
:1024700010E08981081708F008CFF801E25CFD4FF1
:10248000808190913501892331F02D2D4F2D6E2DB6
:10249000C8010E944E070F5F1F4FEBCF85E297E008
:1024A0000E94D90907C08EEF96E0FACF87E198E045
:1024B0000E94D50A9091340121E0290F2093340124
:1024C000811173C482E080933701809136018111BC
:1024D0006CC48D81882309F475C4892F0E940B0672
:1024E00085CE88EF97E0E4CF8DED97E00E94700AEB
:1024F000E1CF82EC97E0FACF8CEF96E0D1CF83EF7B
:1025000096E0CECF8AEE96E0CBCF81ED96E0C8CFB5
:1025100083EC96E0EBCF8CEB98E0CACF81EB97E0B1
:10252000C7CF8DE997E0E2CF86E996E00E941C0ACA
:10253000C1CF88E696E0FACF80E396E0F7CF8091AE
:1025400034010E940B06998390913601911120C0AD
:1025500060916B0520E1620F08F46FEF80915F05D9
:10256000909160050E94E5086AE070E00E94192CD5
:10257000892B61F40E947708A0E48A9FC00111248E
:1025800060913501892F90E00E949E0989817DCE5E
:10259000082F10E0B981EB2EF12C0E151F05B4F7B2
:1025A00060913501C8010E949E090F5F1F4FF5CF52
:1025B000809134010E940B0699839091360191110C
:1025C0001FC060916B0520E1620F08F46FEF8091EE
:1025D0005F05909160050E94E50865E070E00E944B
:1025E000192C892B99F60E947708E0E48E9FC00190
:1025F000112460913501892F90E00E942B0BC6CFEA
:10260000082F10E0F981EF2EF12C0E151F050CF0AC
:10261000BDCF60913501C8010E942B0B0F5F1F4F8A
:10262000F4CF809134010E940B06082F9983E0902B
:102630006905F0906A051091680560916B056695D3
:102640006695669580915F05909160050E94E5080A
:102650000E94350820E8280F27FD2195220F3CE035
:10266000239F212D1124612F620F7E2D8F2D0E941B
:102670001A09F62EE72ED82E10E02981021710F045
:10268000822F03CEF801E25CFD4F808190913501ED
:10269000892331F02D2D4F2D6E2DC8010E944E073C
:1026A0000F5F1F4FEACF84E598E0FACE8FE196E006
:1026B000F7CE809134010E940B06F92E40915F0500
:1026C00050916005609161057091620580911203DF
:1026D00090911303A0911403B091150384179507EB
:1026E000A607B70708F04FC00E94770830E4839F21
:1026F00080011124012F1127F801E25CFD4F808138
:1027000090913501892309F43EC00E94770881FD2C
:102710003CC00E94770889830E94770840E8849F24
:10272000C00111247FE7790F80916A0569810E94B9
:102730001A09462F672F282FC8010E944E072091A3
:102740006B0530E1230F08F42FEF60E1822F90E05A
:102750000E94E508BC0184EF91E00E94192C809151
:102760005F0590916005A0916105B0916205860FAB
:10277000971FA11DB11D8093120390931303A09383
:102780001403B09315038F2D80CD80E070E0198283
:10279000CDCF4091D6035091D7036091D80370916B
:1027A000D90380915F0590916005A0916105B0917A
:1027B000620584179507A607B70708F448CD8091EE
:1027C0003601811150C0809134010E940B069E8316
:1027D000E82EF12C53E0859F800111240A5E1C4FE6
:1027E0002E81E21608F47CC0822F0E940C09811110
:1027F00038C020E04E814150550B7A01822F90E085
:102800008E159F050CF481C00E9477088701000F88
:10281000111F81FF92C00E0D1F1DF801EA5EFC4FD3
:102820001082118212820E94EF0869837A838B835F
:102830009C8380915F0590916005A0916105B091A6
:10284000620529813A814B815C81820F931FA41F0D
:10285000B51F8093D6039093D703A093D803B0936A
:10286000D9038E8112CD40E060E080E00E945107E4
:10287000F6E1EF2EF3E0FF2E10E000E00E94770873
:1028800081FF10C0D7011C9211961C9211971296CD
:102890001C920F5F1F4FB3E0EB0EF11C00341105CB
:1028A00069F791CF0E94770889830E947708B0E882
:1028B0008B9FC00111247FE7790FC801880F991FF2
:1028C000800F911FFC01EA5EFC4F6F0169818091CE
:1028D0006A050E941A09D6016D937D938C93D9CF16
:1028E000F701E25CFD4F808190913501892339F039
:1028F000F801228140816181C7010E944E070D5F6E
:102900001F4FFFEFEF1AFF0A6BCFAC01440F551FAB
:10291000480F591F4A5E5C4F0196FC01EE0FFF1FE6
:10292000E80FF91FEA5EFC4F80819181A281FA01D4
:1029300080839183A2832F5F61CF0E947708D82E76
:102940000E947708F0E88F9FC00111247FE7790F7C
:102950000E0D1F1D0A5E1C4F6D2D80916A050E9491
:102960001A09D8016D937D938C935DCF80913601C8
:10297000882329F040E060E080E00E9451078091C8
:1029800034010E940B06592E40915F05509160055D
:1029900060916105709162058091F2039091F3035B
:1029A000A091F403B091F50384179507A607B70724
:1029B00008F084C0609168057091690580916A058E
:1029C0000E941A096E83772E682E4AEDE42E43E0AA
:1029D000F42E06E811E0580148016701F2E0F9839E
:1029E00002C031E03983D6012D916D01F40181914E
:1029F0004F0190E0222309F463C0262D4E81672DFC
:102A00000E944E07D50116968C91262D4E81672D7A
:102A100090E00E944E07D6018C91F6013197808399
:102A2000B1E0AB1AB108E981E130D9F6D8011296CC
:102A30008C9190E0F7012281222309F44CC0262DCD
:102A40004E81672D0E944E07D80114968C91262D39
:102A50004E81672D90E00E944E070E947708837098
:102A600091E009F090E0D70112969C93B3E0EB0E51
:102A7000F11C095F1F4FE1E00E3B1E0709F0ABCFD1
:102A80000E94EF0869837A838B839C8380915F0522
:102A900090916005A0916105B091620529813A810C
:102AA0004B815C81820F931FA41FB51F8093F2039B
:102AB0009093F303A093F403B093F503852DE5CB36
:102AC00020E040E060E00E944E07F501868120E0B2
:102AD00040E060E09DCF20E040E060E00E944E07D3
:102AE000F801848120E040E060E0B4CF80913401BF
:102AF0000E940B06982EC92E80913601882361F022
:102B000040E060E080E00E945107EBEFF3E088E3F3
:102B1000DF011D928A95E9F780913401811117C078
:102B20008091F7039091F8030E9435049C0181E0A5
:102B30002931310508F480E08093F603293131050D
:102B400030F00E9461049093F8038093F703B12C56
:102B5000A12CD12C97E0792E25E5622E3AEA832E1E
:102B60005524539405C0FCE0FA1508F457C0D12C45
:102B70002D2D30E07B9C80011124F801EA57FE4F97
:102B8000E20FF31FE080E91408F440C0EC1408F0F1
:102B90003DC0A394F12CF701E25CFD4F8081909140
:102BA0003501892309F432C005501C4F020F131F51
:102BB000F801F081F9834F2F262D421B08F440E0E5
:102BC00070916905382D5F2F350F08F43FEF509154
:102BD0006A05232F220F230F2E5F259F212D1124FD
:102BE000682D641B822F0E941A09462F672F282FF9
:102BF000C7010E944E078091F603882339F029818E
:102C0000652D261B08F420E0D8012C93D394B7E05F
:102C1000DB12AECFB394E8E0BE12A5CF8C2D35CB3E
:102C200020916A05298333E0239F800111241695A2
:102C3000079516950795502EA22EB12C8FEF90E098
:102C4000B5010E942D2C762E80913601882371F0DB
:102C500040E060E080E00E945107EBEFF3E088E3A2
:102C6000DF011D928A95E9F71092FA038091F9032A
:102C70008F5F8093F903F12CE12CA01AB10A670150
:102C8000612CD701A550BC4F4D018091FA038629D4
:102C900009F046C00E94AF2C853595400CF040C02D
:102CA0002981F4012083F601EA57FE4FE081EF3FCE
:102CB000D1F0D601A550BC4F2C91F0E0521608F08F
:102CC00041C030E0201B310B209FC001219F900D9F
:102CD000309F900D1124B5010E94192C262F498197
:102CE000CF010E944E07639457E0C50ED11C68E0E7
:102CF0006612CBCF7FEFE71AF70A87E0E816F104F8
:102D000009F0BDCF8091F903781202C01092F90347
:102D10008091FA038F5F8D3100F58093FA0397CA93
:102D2000F601E550FC4F8081882309F4BCCF39813E
:102D3000831708F0B8CF9091F9037912B4CF81507E
:102D40008083B1CF4981429FC0011124B8010E9404
:102D5000192C462F20E060E0C3CF1092FA0325E241
:102D600034E087E042E054E099819150ABEFB3E06A
:102D7000F901873049F4D1966C91D1977981761316
:102D800003C0D1969C93D19760817981671710F029
:102D900090837783119631964A175B0751F78150DC
:102DA000275031098111E2CF52CAAD81AA2309F41B
:102DB0001DCA93CBBD81B0933201237020933101A2
:102DC0000E945C1083E00CCA80916605882351F054
:102DD00048E050E068E170E087E695E00E94F32C5F
:102DE00010926605C0905F05D0906005E090610587
:102DF000F0906205809101058823B9F02FB7F8940F
:102E000080910A0590910B05A0910C05B0910D05DC
:102E10002FBF8C199D09AE09BF094097A105B105C7
:102E200008F4E4C910923701E1C90E946A0BDC0181
:102E3000CB01EFCF9091FB0292FB222720F92817BC
:102E400079F080FB92F99093FB026091FA02709105
:102E5000FB0284E090E00E94212D82E00E94A10EFE
:102E600008958091B8029091AF02892B9091AE02A3
:102E7000992389F0892B90E022E832E0F901408122
:102E80002F5F3F4F41119F5F42E028383407B1F771
:102E900091111092AE028093800248E050E060EB06
:102EA00072E080E892E00E94BF2C892BA9F088E0B4
:102EB000E0E8F2E0A0EBB2E001900D928A95E1F734
:102EC000E0910505F0910605309731F00280F3811D
:102ED000E02D80E892E009950895CF931092B80212
:102EE000C6E0E2E8F2E0DF018C2F1D928A95E9F757
:102EF00090E080E00E94AD0490E080E00E948704B2
:102F00001092AF020E943117EBEFF4E0DF011D9247
:102F1000CA95E9F71092F4041092F5041092F604A1
:102F20000E94E404CF910895AAE2B0E0EAE9F7E153
:102F30000C94F12B8DE195E0FC0101962091F100BC
:102F4000208325E085329207B9F780911E058930EC
:102F500009F456C0C8F4823009F4B2C0833009F4D1
:102F600081C0813071F18091E80083FF7CC2809143
:102F70001D0590911E059A3008F075C2E92FF0E00A
:102F8000E355F24D0C94412C8A3009F488C08B3003
:102F900051F780911D05813231F780912105909183
:102FA0002205892B01F78091E800877F8093E80054
:102FB0000E942B0380911F05809333010E946D179F
:102FC000D2CF80911D05813A71F68091E800877F0C
:102FD0008093E8008091210590912205892B61F46E
:102FE00068E081E195E070E00E94D7038091E800FD
:102FF0008B778093E800B7CF60E090E080E0F3CF7C
:1030000080911D05813209F0AECF8091210590910C
:103010002205029708F0A7CF8091E800877F809370
:10302000E8008091E80082FF18C09091F300809141
:10303000F200029731F48091F100813011F0863076
:1030400021F48091F100809310058091E8008B7746
:103050008093E8000E942B0386CF80911B0581118D
:10306000E0CF81CF80911D05813A09F07CCF80911E
:10307000210590912205892B09F075CF8091E800F8
:10308000877F8093E8008091E80080FFFCCF8091EB
:1030900033018093F1008091E8008E77D9CF809141
:1030A0001D05813209F05FCF8091E800877F809312
:1030B000E8000E942B038091200580930F0553CFD9
:1030C00080911D05813A09F04ECF8091E800877FFD
:1030D0008093E8008091E80080FFFCCF80910F058D
:1030E000D8CF803899F0823809F0BDC18091210590
:1030F0008F70873008F0B7C18093E9008091EB00B2
:1031000085FB882780F91092E90006C08091190597
:1031100090911A05911182609091E800977F9093A9
:10312000E8008093F1001092F1008091E8008E7722
:1031300096C1882309F484C1823009F094C180913A
:103140001F05811187C1809121058F702FEF280FF6
:10315000263008F088C18093E9002091EB0020FF21
:1031600079C1933031F48091EB0080628093EB0061
:1031700071C19091EB0090619093EB0021E030E001
:1031800001C0220F8A95EAF72093EA001092EA0024
:103190008091EB008860EACF811165C110911F0515
:1031A0001F778091E3008078812B8093E3008091EA
:1031B000E800877F8093E8000E942B038091E8005D
:1031C00080FFFCCF8091E30080688093E30082E081
:1031D000111183E080931B0546C18058823008F0AE
:1031E00042C140911F05509120054C3D83E0580796
:1031F000A1F583E08A838AE289834FB7F894DE01E0
:10320000139620E03EE051E2E32FF0E050935700A8
:10321000E49120FF03C0E295EF703F5FEF708E2FC7
:1032200090E0EA30C0F0C7968D939D932F5F2431D4
:1032300059F74FBF8091E800877F8093E8006AE2EA
:1032400070E0CE0101960E94D7038091E8008B7751
:103250008093E80008C1C096E7CF20912105309106
:103260002205852F99278330910509F160F481307B
:10327000910509F472C0029709F0F5C08BE390E064
:10328000EBE2F4E029C08132910509F45AC082973B
:1032900009F0E9C02115310509F469C02130310573
:1032A00009F0E1C08BE790E0ECE6F3E015C0CA015D
:1032B00099274130B1F18230910509F43AC0892B48
:1032C00009F0D1C0E2EBF4E0E4918E2F90E0E2EB64
:1032D000F4E0009709F4C7C02091E800277F20930D
:1032E000E80020912305309124058217930708F404
:1032F0009C0140E02115310509F03EC041113CC060
:103300008091E80082FDA1CF80911B05882309F4FC
:103310009CCF853009F499CF8091E80083FFF0CFEE
:1033200094CFE0E9F4E0E4918E2F90E0E0E9F4E05E
:10333000D0CFE8E7F4E0E4918E2F90E0E8E7F4E006
:10334000C8CF2115310571F02130310509F08BC04E
:1033500089E090E0E6E5F4E0BFCF82E190E0E6E6C8
:10336000F4E0BACF89E090E0EDE3F4E0B5CF84E497
:1033700090E0E7EEF3E0B0CF80911B05882309F4DD
:1033800064CF853009F461CF8091E80083FD5DCF83
:103390008091E80082FDB4CF8091E80080FFAACF41
:1033A0009091F3008091F2002115310519F08830D9
:1033B000910550F041E0089709F040E08091E80065
:1033C0008E778093E80096CF44914093F100319638
:1033D000215031090196E8CF803809F044C080912E
:1033E000E800877F8093E80080911C058093F100BE
:1033F0009CCE811138C010911F051230A0F580912C
:10340000E800877F8093E80010931C050E942B033F
:10341000112311F084E005C08091E30087FDFACF0D
:1034200081E080931B0542E061EC81E00E944A0349
:1034300042E261EC82E00E944A0380911B0513C0C6
:1034400080911F05813079F481E0933009F080E0AC
:1034500080931A051092E9008091E800877F80939D
:10346000E8000E942B038091E80083FF0AC080914E
:10347000E800877F8093E8008091EB008062809372
:10348000EB00AA96E3E00C940D2C0E946D172FEF31
:1034900084E39CE0215080409040E1F700C00000B0
:1034A00088E19AE00FB6F894A895809360000FBE6B
:1034B00090936000FFCF882321F00E94C40D0E94EA
:1034C00031170895882339F09091B802892B8093A1
:1034D000B8020E94311708958823D1F19CEF980F0C
:1034E000913A78F4E2E8F2E09191891303C0DF01A8
:1034F00011971C9292E0E838F907B1F70E94311752
:10350000089590E2980F983050F4877091E001C0D0
:10351000990F8A95EAF7892F0E94C40DEFCF9BE59A
:10352000980F933028F490E080E00E94AD04089555
:1035300098E5980F9B3128F490E080E00E94870482
:10354000089593E3980F933118F460E00E94F40E0D
:103550000895CF93C82F8823A9F08CEF8C0F813A60
:1035600000F5E2E8F2E0DF018D91C81769F022E092
:10357000A838B207C9F76C2F80E892E00E946D046A
:103580000E943117CF9108958191C81303C0DF01C4
:1035900011971C9232E0E838F307B1F70E94311717
:1035A000EACF80E28C0F883068F4C77021E030E009
:1035B00001C0220FCA95EAF78091B802822B80934E
:1035C000B802DECF8BE58C0F833038F42C2F2452D9
:1035D000330BC9010E94AD04D5CFE8E5EC0FEB3108
:1035E00050F4F0E0EE0FFF1FE55CFE4F808191810B
:1035F0000E948704C7CF83E38C0F833118F661E004
:103600008C2F0E94F40EBECFFF920F931F93CF9387
:10361000DF93C62FD42F122FFC0185818823A9F0B8
:10362000609365050E94610490936405809363052F
:10363000C77081E001C0880FCA95EAF70E94621A3C
:10364000CDB7DEB7E5E00C940B2C809165056813CF
:1036500033C080916305909164050E943504883CD5
:10366000910550F500E20D0FCD17A9F0C770FF24AA
:10367000F3948F2D01C0880FCA95EAF70E945B1A58
:10368000083048F48D2F877001C0FF0C8A95EAF747
:103690008F2D0E94621A812F0E94A91A812F0E94E9
:1036A0006C1A083068F6D77081E001C0880FDA958F
:1036B000EAF70E945B1AC4CFC77081E001C0880F8F
:1036C000CA95EAF7F6CFB0E0A0E0E9E6FBE10C949A
:1036D000E92B8C01FC018481882341F121E04081A8
:1036E00051816281738195810E94D80FEC01FC01A8
:1036F000E851FC47E730F105A8F5E954F24D0C9488
:10370000412C26E241EE61EEC8010E94041B80912B
:10371000AD02877059F0F8018581882339F08091D6
:10372000FB0282FF03C082E00E94A10ECDB7DEB78C
:10373000EBE00C94052C27E245EE65EEE5CF26E2A2
:1037400041EE60EEE1CF27E245EE64EEDDCF26E20A
:1037500041EE62EED9CF27E245EE66EED5CF28E204
:1037600041E0EBCFF8018581882309F4F0C3109282
:103770006505CE019057839708F0D3C384E090E0AD
:103780000E94ED2C9093FB028093FA02FE01E1501F
:10379000F047E232F10520F4E254F24D0C94412C52
:1037A0008091FA0281608093FA026091FA0270912E
:1037B000FB0284E090E00E94212D0E946D17A7CFAC
:1037C0008091FB0288608093FB02EFCF8091FA0228
:1037D0008260E9CF8091FA028460E5CF8091FA029D
:1037E0008860E1CF8091FB028160EDCF8091FB0288
:1037F0008260E9CF8091FA028061D5CF8091FA0290
:103800008062D1CF8091FA028064CDCF0E946D1783
:103810008091FA028068C7CF8091FA028C60C3CF92
:103820008091FB028360CFCF8091FA028E7FBBCF65
:103830008091FB02877FC7CF8091FA028D7FB3CF43
:103840008091FA028B7FAFCF8091FA02877FABCF56
:103850008091FB028E7FB7CF8091FB028D7FB3CF2B
:103860008091FA028F7E9FCF8091FA028F7D9BCF4D
:103870008091FA028F7B97CF0E946D178091FA0298
:103880008F7791CF8091FA02837F8DCF8091FB0259
:103890008C7F99CF8091FA0282FB992790F921E0E1
:1038A000922790FB82F990FB83F97DCF8091FB02F8
:1038B000982F909591708E7F892B90FB81F983CF03
:1038C0009091FA02892F8F7B96FF80646CCF0E94C3
:1038D0006D179091FA02892F97FB87F9805863CF73
:1038E00061E08EE090E00E94032D5FCF60E0F9CFB1
:1038F0009091FA02892F8F7E94FF806154CF90912E
:10390000FA02892F8E7F90FF81604DCF9091FB024C
:10391000892F877F93FF886056CF85E321C38091ED
:10392000670591E0892780936705109237018091A0
:103930006605816080936605EACE44EF55E060E05D
:1039400076E00E945A05E3CE40E056E064EF75E071
:10395000F8CF40EE55E06AEE75E0F3CF4AEE55E061
:1039600060EE75E0EECF46EC55E063ED75E0E9CF33
:1039700043ED55E066EC75E0E4CF4CEA55E069EBC9
:1039800075E0DFCF49EB55E06CEA75E0DACF40E94E
:1039900055E06EE975E0D5CF4EE955E060E975E098
:1039A000D0CF81E00E947A02B2CE85E0FBCF8DE0DD
:1039B000F9CF82E1F7CFCB35FCE7DF0708F05FC036
:1039C000C1302CE7D20709F48EC0C3308CE7D8078A
:1039D00009F483C0C115DC4709F463C0F80185818F
:1039E000E080F180882309F482C0C7010E94D60DCF
:1039F000C82F682FC7010E944C0EB7018C2F0E9460
:103A00008E0C0E94AC0CD82FC92F982EF801B580CF
:103A1000A680A2942FE0A2228091AD02877009F1C6
:103A2000DB2CBB20F9F0892F807F803469F080E2A5
:103A30008D0F8830B0F0892F807E803229F4F1E03C
:103A4000FD1778F4AA2069F08091FB0282FF09C07B
:103A500082E00E94A10E8091AD028770DD24D39494
:103A60008111D12C8C2F82958F70E82EF12C8C3007
:103A700008F0A2C0F701E052F24D0C94412CCB3576
:103A8000ECE7DE0791F1CC35DC4709F0A7CF809158
:103A9000FB0282FB882780F991E089270E941A1790
:103AA0009DCF0E946D172FEF84E39CE02150804052
:103AB0009040E1F700C0000087E797E79093010886
:103AC0008093000888E19AE00FB6F894A895809357
:103AD00060000FBE90936000FFCF6FEF7FEF90E02C
:103AE00080E00E94212D0E94451A80E0D7CFC701B7
:103AF0000E94190EC82F81CF2C2F2F70C22EC07F8D
:103B000019F0C29490EFC9228D2FBB20B9F0CC20C0
:103B100069F090E29D0F983010F0D11109C08091AA
:103B2000B802C82AC092B8020E9431178D2F42C035
:103B30008091AF02C82AC092AF02F6CF0E946C1AE1
:103B4000CC20D1F1D05ED83010F0911004C08C2D73
:103B50000E94C40D06C0C0948091AF02C822C092DA
:103B6000AF020E94311728C08C2F8F70C82EC07FE3
:103B7000C03219F0C29480EFC822992059F091E028
:103B8000991609F47AC0BB2009F486C0AA2009F46A
:103B900048C0CCCF8091FB0282FD3FC0BB20B9F171
:103BA000CC2039F08091B802C82AC092B8020E9495
:103BB000311780E00E94A91AE8E0EE1AF108F4E05B
:103BC000EF16F10410F40E94D304DD20A9F08091D7
:103BD000AD0280FD11C0F801158286958695869507
:103BE0000E94B80EC8010E94631B8091AD028695A9
:103BF000869586950E948F0E20E0F80140815181C4
:103C000062817381848195810E94D80F8FCD80E07D
:103C10000E946C1ACC2081F29ACFBB20A1F0A11097
:103C200004C08C2D0E94621AC7CFE1E0AE12C4CF4F
:103C30008091AE029C2D9823C91609F4BDCFC82AE5
:103C4000C092AE02B9CFA110B7CF8C2D0E945B1AE3
:103C50009091AE028C2D892329F08C2D809589239B
:103C60008093AE02809189029C2D982309F4A4CF01
:103C7000C094C822C09289029FCFBB2029F0F5E0F2
:103C8000FA1508F499CFCDCF24E02A1508F494CF83
:103C90008C2D0E945B1A90CFAA20D1F3D93349F41E
:103CA0008FEF97EEE3E081509040E040E1F700C0F5
:103CB00000008D2F0E946C1A7FCF8C2F86958695E1
:103CC000837069F0813009F077CF8D2F9C2F93702E
:103CD000B11002C080E090E00E9487046DCF8D2F6C
:103CE0009C2F9370B11002C080E090E00E94AD0460
:103CF00063CF6B2D8D2F0E94F40E5ECF8C2F8370BF
:103D000009F040C0B11058CF4D2F429546954770ED
:103D1000440F440F2D2F2F7030E0042E02C0220FCD
:103D2000331F0A94E2F790E080E0D4FF09C08FE0EF
:103D300090E002C0880F991F4A95E2F78095909510
:103D4000C695C695C370C230A1F0C33079F04091DA
:103D5000F6025091F702C13039F0822B932B842365
:103D600095230E94C80E28CF242B352B822B932B12
:103D7000F8CF822B932B2091F6023091F702822705
:103D80009327EFCF8695BB2011F08C2F817088236D
:103D900009F412CF4D2F429546954770440F440FBA
:103DA0002D2F2F7030E0042E02C0220F331F0A94F3
:103DB000E2F790E080E0D4FF09C08FE090E002C01D
:103DC000880F991F4A95E2F780959095C695C695FC
:103DD000C370C230A1F0C33079F04091F802509125
:103DE000F902C13039F0822B932B842395230E9452
:103DF000820EE2CE242B352B822B932BF8CF822BF5
:103E0000932B2091F8023091F90282279327EFCF6C
:103E1000CF70BB2029F08C2F0E94B80E8D2F02CFBF
:103E20008D2F0E945B1A8C2F0E948F0EC5CE8D2F76
:103E3000F2EF9F1699F1F91570F020EF9216D1F07C
:103E400091EF991691F0BB2009F45BC0A1106ECEE2
:103E50008C2F8F7127C0E3EF9E1639F1F4EF9F127C
:103E6000F2CF8091FB0282FD2EC08C2F8F71BB2080
:103E7000D9F218C0BB2069F024E02A1508F49CCEC2
:103E8000CF7181E090E002C0880F991FCA95E2F7D8
:103E9000B8CF85E08A1508F48FCEF2CF8C2F8F71C2
:103EA000B110C2CF0E94B80E87CE90E080E0BB2058
:103EB00009F49DCFCF7181E090E002C0880F991F77
:103EC000CA95E2F794CFBB2089F0CF718C2F0E9466
:103ED000B80E8091FB0282FF07C0E8E0CE9FC001D0
:103EE000112483608093AD028C2FDCCF81E00E948F
:103EF000A10EF1E0FA1508F05FCE82E00E94A10E5B
:103F00005BCEAA2059F0893309F0D3CE2FEF87EE8C
:103F100093E0215080409040E1F7C9CE8C2F8F7103
:103F200083CFC631FCE7DF0749F58091B8028A7A72
:103F300091E009F490E09093880269E2811165E3D1
:103F400080E892E00E946D040E943117E0CBC631F8
:103F50002CE7D207D1F4809188028111DECC89E26E
:103F6000E2E8F2E028E832E09191891303C0DF0132
:103F700011971C922E173F07B9F7E6CFCA358CE789
:103F8000D80709F018CD81E089CD8091B8028272FE
:103F9000FE01E052F847E531F10508F01FCDE4518C
:103FA000F24D0C94412CCF93DF938091AC02807F33
:103FB00009F04DC08091AB02882309F448C0E0911C
:103FC0005E0550912505C091A702D091A60260918F
:103FD000A8027091A90247E05E17C9F18E2F90E008
:103FE000E49FF0011124EA5DFA4F2481222391F12C
:103FF000489FF001499FF00D1124DF01AA5DBA4FDF
:1040000011962C9111972C1325C02C912D1322C0A1
:1040100015962C91159721111DC012962D913C914A
:10402000261B370B283C3105A8F48091AC028F7019
:1040300080618093AC02E45DFA4F80818F70806173
:10404000808386EA92E00E94631B0E94CC0DDF9180
:10405000CF910895FC013196E770BECFADE0B0E09E
:10406000E4E3F0E20C94E82B8C0186E0F801DE0139
:10407000189601900D928A95E1F7F8018481E58008
:1040800096EAA92E92E0B92E9091AA02911128C029
:10409000882319F1EE20F1F0C8010E94CD0EF82E10
:1040A0008823C1F087E0F801D50101900D928A952F
:1040B000E1F78091AA02813031F48091A6029091BB
:1040C000A7020E940A0E0E94D31F8F2D2D96ECE0AE
:1040D0000C94042CC8010E94631BFF24F394F5CFB9
:1040E000D080C18082809380F090AB022091A802A2
:1040F0003091A902A401421B530BFF2009F4BCC05C
:10410000483C510508F092C08823F9F29091A7022B
:104110008091AC02282F207F09F056C0C91214C02C
:104120009091A602D91210C0E11048C08F70806132
:104130008093AC0286EA92E00E94631B8091AC02FD
:10414000F8018683F12CC1CFE11038C06C2D8D2D84
:104150000E9493026C2D8D2D0E949302E82E8111F6
:10416000F1CFD886C986888599850E940A0E292FA5
:1041700022952F70903458F49F70223088F0992344
:1041800099F0F8019681907F79F4FE2C9ECF2A5FFA
:104190002F70223068F0C8010E94631BEF2CF5CF0E
:1041A000992311F0882389F3805E883070F3F3CF70
:1041B000803F58F3815F833040F3EDCF8091AC02B4
:1041C00081608093AC02BECFC91207C09091A60255
:1041D000D91203C0EE2009F470C0C8010E94CD0EB0
:1041E000882309F477CFEE2009F474CF8091AC02D4
:1041F000803288F02091A6023091A7023A83298369
:104200009C828B829091AA029D831E828F83CE0115
:1042100001960E94631B87E0F801A6EAB2E00190D4
:104220000D928A95E1F70E94D31F57CF9091AC026F
:10423000292F207F51F486EA92E00E94631B87E0D9
:10424000F50111928A95E9F77DCF882309F43DCFD6
:104250008091A7028C11C1CF8091A602D812BDCF48
:10426000E110BBCF9683C8010E94631B87E0F50174
:1042700011928A95E9F729CF483C5105B8F7882370
:1042800009F42BCFFE2CEE2009F424CF8091A70255
:104290008C1120C08091A602D8121CC08091AC0263
:1042A00080FD0FC0982F907F61F08683903F31F0A2
:1042B000982F907F905F8F70892B8683C8010E9412
:1042C000631B87E0F801A6EAB2E001900D928A959F
:1042D000E1F7FBCEC8010E94CD0E81119CCF8091E9
:1042E000AC0281608093AC02C8010E94631BEDCEDA
:1042F000ABE1B0E0EEE7F1E20C94F02B4E8B5F8B7C
:10430000688F798F8A8F192F9B8F91111092AF022E
:104310001D8A86E0FE017696DE011F9601900D92C1
:104320008A95E1F70A8D002341F021E04F855889F5
:1043300069897A89C8010E94D80F0B8B1C8B87E092
:10434000FE013F96DE01189601900D928A95E1F7E5
:10435000CE0108960E942E2081110CC087E0FE013C
:104360003896DE01119601900D928A95E1F74C8501
:1043700041110BC017E080915E05909125058913CE
:1043800032C06B96E4E00C940C2C2091250530E0B3
:10439000C90101968770992750915E055817190633
:1043A000A1F04D8397E0929FD001939FB00D11240F
:1043B000AA5DBA4FFE01319601900D929A95E1F7F0
:1043C000809325050E94CC0DD5CF0E946D171092C9
:1043D000250510925E0587E0E6EAF2E0DF011D9216
:1043E0008A95E9F7C7CF819FC00111248A5D9A4F52
:1043F0000E942E20882329F280915E0590E001968C
:104400008770992780935E05B6CFA6E0B0E0EBE019
:10441000F2E20C94F02B0E9461048C018091B902AD
:104420009091BA028017910781F019821A820E9436
:104430006104682F49815A81792F80E090E00E94C1
:1044400078211093BA020093B9022696E4E00C9406
:104450000C2CA8E0B0E0EFE2F2E20C94F12B4091DA
:10446000CD025091CE026091CF027091D0022FB751
:10447000F89480910A0590910B05A0910C05B091DC
:104480000D052FBF841B950BA60BB70B11E08436CF
:104490009105A105B10578F10E946A0BDC01CB0101
:1044A0000296A11DB11D89839A83AB83BC83809141
:1044B0001501909116018F529D4F20911401422FAA
:1044C00050E0253010F044E050E0BE016F5F7F4FB8
:1044D0000E94CC2C82E090E00E946C2B182F882345
:1044E00051F00E9444046093CD027093CE028093F9
:1044F000CF029093D002812F2896E3E00C940D2CEC
:10450000A9E0B0E0E6E8F2E20C94F12B88E0E7E6FF
:10451000F5E0DE01119601900D928A95E1F719867A
:1045200049E050E06AED72E0CE0101960E94BF2C96
:104530009C014091E3025091E4026091E502709188
:10454000E602EFB7F89480910A0590910B05A091CF
:104550000C05B0910D05EFBF841B950BA60BB70B97
:1045600084369105A105B10518F411E0232B21F142
:1045700080911D0190911E018F529D4F20911C0131
:10458000422F50E02A3010F049E050E0BE016F5F4A
:104590007F4F0E94CC2C83E090E00E946C2B182F60
:1045A000882351F00E9444046093E3027093E40274
:1045B0008093E5029093E602812F2996E3E00C9424
:1045C0000D2CEF92FF921F93CF93DF9300D000D07A
:1045D0000F92CDB7DEB77B0190E080E00E946C2B9C
:1045E000182F882309F487C080910701482F50E0D5
:1045F000882311F041E050E06091080170910901B9
:104600006F527D4FCE0105960E94CC2C4091C9027D
:104610005091CA026091CB027091CC022FB7F894EE
:1046200080910A0590910B05A0910C05B0910D05A4
:104630002FBF841B950BA60BB70B84369105A105E4
:10464000B10540F482ED92E00E94B1029D8189178C
:1046500009F451C081E090E00E946C2B81111AC0D6
:1046600010E08091C5029091C602A091C702B0915E
:10467000C802F70180839183A283B383812F0F90B7
:104680000F900F900F900F90DF91CF911F91FF909F
:10469000EF90089580910F01482F50E0853010F081
:1046A00044E050E060911001709111016F527D4F14
:1046B000CE0101960E94CC2C82ED92E00E94B102C4
:1046C0009D818913CDCF0E9444046093C9027093E9
:1046D000CA028093CB029093CC0289819A81AB81EC
:1046E000BC818093C5029093C602A093C702B09389
:1046F000C80211E0B6CF8091D2029091D302A0916E
:10470000D402B091D50289839A83AB83BC83111103
:10471000E4CFA7CFA0E1B0E0E0E9F3E20C94E82B0E
:104720001A821982FE01339686E0DF011D928A9576
:10473000E9F783E7A82E81E0B82E10E000E0EE2430
:10474000E394F12C2EE7C22E21E0D22EF5018191C7
:104750005F018F3F09F445C0F894E82FE295EF70B0
:10476000F0E021A18F70A70102C0440F551F8A9568
:10477000E2F7CA01922F982B91A392A180958923E9
:1047800082A3789400C0E7E7F1E031E0912C219119
:104790002F3F09F49DC0A22FA295AF70B0E0909674
:1047A0008C9190E02F7002C0959587952A95E2F73D
:1047B00080FD8EC0832F982A330FCE16DF0639F77F
:1047C000F501319780818F3F11F00E94510B50EA23
:1047D0005A95F1F7E1E0F0E0EC0FFD1FE00FF11F5B
:1047E00090820F5F1F4F0430110509F0AFCF48E0F2
:1047F00050E0BE016F5F7F4F8CEE92E00E94BF2CB5
:104800009C01892B49F088E0FE013196ACEEB2E0C4
:1048100001900D928A95E1F70091F50210E00450A5
:104820001D4F232B09F456C081E08093BD020E94E6
:1048300061049093BC028093BB02F12CE0900105CF
:10484000EE2009F4A1C01A8619861C861B86809169
:10485000E7028A3008F062C041EE52E2BE01675FB3
:104860007F4FC8010E948910882309F47CC049E267
:1048700052E2BE01675F7F4FC8010E948910882302
:1048800009F471C040E852E2BE01675F7F4FC80182
:104890000E948910882309F466C01092E702809173
:1048A000F40290E044E050E0BE01675F7F4F845027
:1048B0009D4F0E94BF2C21E02093C402892B09F058
:1048C00044C0E12C8E2D8F296096ECE00C94042CD2
:1048D00080E071CFF090BD02FF2009F4AECF80914F
:1048E000BB029091BC020E943504059708F4A5CF45
:1048F00044E050E06CEE72E0C8010E94BF2C892BAE
:1049000059F084E0ECEEF2E0D80101900D928A9526
:10491000E1F71092BD0292CFF12CFBCF8091BE0245
:104920009091BF020E943504843F914008F094CFDB
:104930008091C402882329F2FE01399684E0DF01C8
:104940001D928A95E9F71092C402E091F402F0E01A
:10495000E450FD4F89859A85AB85BC858083918322
:10496000A283B383AFCF8091E7028F3F31F08F5F97
:104970008093E7028A3008F492CF0E9461049093FA
:10498000BF028093BE02D4CFF80180819181A281C1
:10499000B3818093D2029093D302A093D402B093B8
:1049A000D50282ED92E00E94B1028093D102809004
:1049B000D6029090D702A090D802B090D9028091F0
:1049C000C0029091C102A091C202B091C3028816A8
:1049D0009906AA06BB06B1F08092C0029092C1026D
:1049E000A092C202B092C3020E944404861A970A9F
:1049F000A80AB90A8092E8029092E902A092EA021B
:104A0000B092EB0288E0EAEDF2E0A7E6B5E00190B3
:104A10000D928A95E1F756CF1F920F920FB60F9223
:104A200011242F933F934F935F936F937F938F93B3
:104A30009F93AF93BF93CF93DF93EF93FF93D09167
:104A4000E900DF708091EC00C82FC17080FDC0E8E4
:104A50001092E9008091F000877F8093F0007894B5
:104A60000E9494171092E9008091F0008860809372
:104A7000F000CD2BCF70C093E900FF91EF91DF9153
:104A8000CF91BF91AF919F918F917F916F915F91E6
:104A90004F913F912F910F900FBE0F901F9018953F
:104AA0001F920F920FB60F9211242F933F934F93A3
:104AB0005F936F937F938F939F93AF93BF93EF9386
:104AC000FF938091E10082FF09C08091E20082FFA4
:104AD00005C08091E1008B7F8093E1008091DA0036
:104AE00080FF24C08091D80080FF20C08091DA0030
:104AF0008E7F8093DA008091D90080FF9BC080E197
:104B000089BD82E189BD09B400FEFDCF81E08093BB
:104B10001B0580910E05811109C00E94DB020E94D5
:104B20007C038091E20084608093E2008091E10048
:104B300080FF17C08091E20080FF13C08091E200E7
:104B40008E7F8093E2008091E20080618093E2009A
:104B50008091D80080628093D80019BC85E0809352
:104B60001B058091E10084FF29C08091E20084FF51
:104B700025C080E189BD82E189BD09B400FEFDCF79
:104B80008091D8008F7D8093D8008091E1008F7E46
:104B90008093E1008091E2008F7E8093E20080911B
:104BA000E20081608093E20080911C05882309F473
:104BB00047C084E080931B0580911B058091E10034
:104BC00083FF27C08091E20083FF23C08091E10032
:104BD000877F8093E10082E080931B0510921C0583
:104BE0008091E1008E7F8093E1008091E2008E7FD2
:104BF0008093E2008091E20080618093E20042E0D5
:104C000060E080E00E944A038091F0008860809319
:104C1000F000FF91EF91BF91AF919F918F917F91A4
:104C20006F915F914F913F912F910F900FBE0F9019
:104C30001F90189519BC10921B0510920E0576CF87
:104C40008091E30087FD02C081E0B4CF83E0B2CF62
:104C500078941F921FB61F9211248F939F93AF9346
:104C6000BF9380910A0590910B05A0910C05B0911E
:104C70000D050196A11DB11D80930A0590930B05AA
:104C8000A0930C05B0930D05BF91AF919F918F91AB
:104C90001F901FBE1F9018951F921FB61F921124C0
:104CA0008F939F93AF93BF9380910905811113C098
:104CB00080910A0590910B05A0910C05B0910D050E
:104CC0004196A11DB11D80930A0590930B05A093F9
:104CD0000C05B0930D05BF91AF919F918F911F90DF
:104CE0001FBE1F901895CDB7DEB762970FB6F89428
:104CF000DEBF0FBECDBF85B7806885BF85B7806832
:104D000085BF84B7877F84BF0FB6F894A89580913C
:104D10006000886180936000109260000FBE80E8A0
:104D200090E00FB6F89480936100909361000FBEFD
:104D30008FE49BE090937F0280937E020E94DB02CF
:104D40000E947C038091E20084608093E20078946A
:104D500080911B058823A1F01091E9001F709091AC
:104D6000EC00892F817090FD80E8182B1092E900EB
:104D70008091E80083FD0E9494171F701093E90052
:104D800082E084BD93E095BD9AEF97BD80936E005D
:104D90001092E8021092E9021092EA021092EB02DD
:104DA0008091D80080618093D8002AE12A95F1F79C
:104DB00000C08091D900182F117080FD04C00E949E
:104DC000DB0210921B05109301051093020510934E
:104DD000240111110E947F2A8091240180912401D5
:104DE00094E0811190E09093F50284E0891B809318
:104DF000F40284E90E94510B86E60E94510B87E978
:104E00000E94510B86EC0E94510B07E711E05EE710
:104E1000E52E51E0F52ED8018D918D018F3F11F0D7
:104E20000E94510BE016F106B1F788E0ECEFF2E0DA
:104E3000DF01282F1D922A95E9F7ECEEF2E0DF0161
:104E40001D928A95E9F790E080E00E94ED2C863E65
:104E50009E4F09F466C066EE7EEF90E080E00E940F
:104E6000212D60E082E090E00E94032D81E090E03F
:104E70009093F7028093F60261E083E090E00E9455
:104E8000032D60E074E184E090E00E94212D60E059
:104E900086E090E00E94032D60E087E090E00E94B1
:104EA000032D40E050E0BA0188E090E00E94152D0B
:104EB00060E084E290E00E94032D60E087E190E0F2
:104EC0000E94032D60E08CE090E00E94032D60E0E2
:104ED0008DE090E00E94032D19821A821B821C82B1
:104EE0001D821E821F82188648E050E068E170E053
:104EF000CE0101960E94F32C40E050E0BA0180E21E
:104F000090E00E94152D40E050E0BA018FE090E063
:104F10000E94152D40E050E0BA0183E190E00E942C
:104F2000152D82E090E00E94E52C8093040384E03C
:104F300090E00E94ED2C9093FB028093FA0283E0B4
:104F400090E00E94E52C90E00E94C80E0E948D0522
:104F500081E08093660548E050E068E170E087E614
:104F600095E00E94D52C10926605809167058C7F94
:104F7000F9F485E3809367058091380190913901B8
:104F8000A0913A018093680590936905A0936A0502
:104F90008FE780936B058FEF80936C0548E050E0BE
:104FA00068E170E087E695E00E94F32C10926605B8
:104FB00080910105811102C00E94822A85E291E060
:104FC000909306058093050580911B0500E112E191
:104FD000853009F4E1C00E948A2345E053E05A87F6
:104FE00049878CEF92E09C878B872DE033E0DC01D2
:104FF000FA0191918D912E173F0709F4D7C09817A8
:10500000C1F320900105912C812C10E0AB85BC856B
:105010007D90BC87AB87E985FA855190FA87E9874F
:10502000571409F476C05724740100E06624639491
:10503000852D862109F461C0D72CD6202220A1F02D
:1050400009831A830E9461049C838B83F1E0FD83B2
:1050500091E0D11001C090E09E8349815A816B811B
:105060007C818D810E947821DD2009F446C08091E9
:1050700067058C7F8C3709F040C0F701EA57FE4F77
:1050800080818F3F09F439C0B12CA12C312C90E0E4
:105090009C01220F331FA90142545E4F588B4F874A
:1050A000D901A154BE4FBA8BA98BF701E550FC4F33
:1050B000FE87ED876501412CF601EA57FE4F80819E
:1050C0008F3F61F031125EC140125CC1AD85BE857B
:1050D0002C9130E2230F08F42FEF2C934394FFEF31
:1050E000CF1ADF0A27E04212E7CF339437E0A30E4E
:1050F000B11C48E3A416B104E9F60F5F660C5FEF3C
:10510000E51AF50A073009F093CFE985FA8531975A
:1051100070821F5F87E0880E911C183009F076CFEF
:105120000E946A0B47C080911B05843031F10E94B8
:10513000C21010920905E8E1F0E020E40FB6F894FF
:10514000A895E09360000FBE2093600083B7817F35
:10515000846083BF83B7816083BF7894889583B769
:105160008E7F83BF0FB6F894A89580916000886108
:1051700080936000109260000FBE80911A05882312
:1051800059F00E948A23ECEFF2E0819181113DC138
:1051900033E0E430F307C9F780911B05853009F44B
:1051A000C2CF0E946D170E94D30415CF981329CF48
:1051B0000E9405220E94C21086E0EBEFF4E0DE01BF
:1051C000119601900D928A95E1F7D090FC04F09031
:1051D000FD040091FE04E090FF0410910005109280
:1051E000FD041092FE041092FF0410920005802F1F
:1051F0008F2909F445C08091F9049091FA040E9426
:1052000035049C018091F404882309F419C12531E7
:105210003105B0F18F3F19F08F5F8093F404FF20C8
:1052200059F00E942C059FEF1F140CF491E0899F08
:10523000802D11248093FD04002359F00E942C0539
:1052400091E010160CF09FEF899F802D1124809320
:10525000FE048091FD04882399F0C090FE04CC20C8
:1052600079F00E944C05882309F4C7C08093FD049F
:105270008C2D0E944C05882309F4C1C08093FE0444
:10528000812F8E2909F445C08091F7049091F8048C
:105290000E9435049C018091F504882309F4CBC059
:1052A00021353105B0F18F3F19F08F5F8093F50400
:1052B000EE2059F00E940A059FEF1E140CF491E0B5
:1052C000899F802D11248093FF04112359F00E949F
:1052D0000A0591E011160CF09FEF899F802D112493
:1052E000809300058091FF04882399F0C090000509
:1052F000CC2079F00E944C05882309F482C0809369
:10530000FF048C2D0E944C05882309F47CC08093F7
:1053100000058091FC04D81219C08091FD048823F7
:1053200011F08F1113C02091FE04222311F00213FB
:105330000DC090910005992311F0191307C0309109
:10534000FF04311103C0822B892B11F00E94E40469
:10535000DA82FB820C83ED821E8386E0FE013196A9
:10536000ABEFB4E001900D928A95E1F70E94D3046F
:1053700090910D03891709F427CE80930D030E94A5
:10538000440422CE90E0AF85B8894C91FC01EE0F29
:10539000FF1FE254FE4F2081421B550BE989FA8919
:1053A0002081880F991FFC01EA57FE4F81AD281B11
:1053B000330B449FB001459F700D700D1124229F47
:1053C000C001239F900D900D1124860F971F0E94FE
:1053D0008C08382F893208F081CE28E2231B08F48C
:1053E00020E0F601E550FC4F213108F020E130814A
:1053F000320F08F43FEF308371CE81E037CF81E088
:105400003DCF81E07CCF81E082CF09BD19BD09B4D9
:1054100000FEFDCF8091D8008F7D8093D8008091D1
:10542000E00082608093E0008091E00081FDFCCF8D
:105430000E946D17B1CE2B30310508F036CF69CF01
:105440002B30310508F0E8CE1BCF8EE14B9B02C01C
:105450008150E1F74B9BFECF08955B9880E28A95DF
:10546000F1F75B9A0895FC013BE03A95F1F798E07B
:1054700020E080E031E040E14A95F1F7880F4B9B56
:1054800002C08160232742E04A95F1F7000040E125
:105490004A95F1F7915079F790E19A95F1F799B122
:1054A00032E03A95F1F7000040E14A95F1F793FBBD
:1054B000992790F992272081920F90830895A1E077
:1054C000B0E0E5E6FAE20C94EE2B19828C017C0147
:1054D000E60EF11C0E151F0541F481E09981911132
:1054E00080E02196E6E00C940A2C0E94252ACE0149
:1054F00001960E94332AF80181938F01EBCF539AD2
:105500005B9A089553985B9AEB9AE9E6F0E0808104
:105510008F73808308956150770B91E001C0990FDC
:105520006A95EAF720E031E0911108C0222391F05A
:105530005B9A80E28A95F1F75B980895492F48239A
:1055400039F05B9A232740E24A95F1F79695ECCF24
:105550005B98F9CF5B98EDCFFF920F931F93CF939A
:10556000DF93EC018C01060F111DC017D10729F440
:10557000CDB7DEB7E5E00C940B2CF9900E942D2AF4
:1055800068E08F2D0E948B2AF0CF1F920F920FB6EA
:105590000F9211240F931F932F933F934F935F9379
:1055A0006F937F938F939F93AF93BF93EF93FF93EB
:1055B000CF93DF930F92CDB7DEB719820E94252AD1
:1055C000CE0101960E94332A282F082F06950695B2
:1055D0000695982F92959570802F8570980F892F3A
:1055E000837096959695890F822787709981892B6C
:1055F00009F05CC0053008F059C080E18A95F1F7E8
:105600005B9A539A82E08A95F1F700C05B9888E034
:10561000089F80011124D801AC5FBE4F1696ED9112
:10562000FC9117973097A9F0609171017091720108
:1056300014962D913C911597260F371F11968D9139
:105640009C911297680F791F13964C9113978C9128
:105650000995F801EC5FFE4F6381662351F02091BC
:1056600071013091720184819581820F931F0E9494
:10567000AC2A0E942D2A80E18A95F1F75B98539815
:105680005B9A80E18A95F1F7F801EC5FFE4F60814B
:10569000662351F0209171013091720181819281D4
:1056A000820F931F0E945F2A0E94252A0F90DF918C
:1056B000CF91FF91EF91BF91AF919F918F917F918A
:1056C0006F915F914F913F912F911F910F910F908B
:1056D0000FBE0F901F9018950F931F93CF93DF93DA
:1056E000EC0105970CF04CC0F894539A5B9885E058
:1056F0008A95F1F700008C2F869585709C2F957008
:10570000890F982F93708695869523E0CC0FDD1F27
:105710002A95E1F7890F8E01082B0E942D2A00C0DF
:1057200068E0802F0E948B2A80E18A95F1F75398D8
:105730005B9A4B9B1EC087E090E04B991CC0FE011A
:10574000EC5FFE4F63816623F9F020917101309187
:10575000720184819581820F931F0E945F2A8111BB
:1057600013C0539A5B9A7894DF91CF911F910F9158
:10577000089500C0DECF019729F4539A5B9A78947C
:1057800080E0F2CF00C0D9CF0E94252A80E28A951E
:10579000F1F75B98539A80E18A95F1F7CC5FDE4F81
:1057A0006881662351F020917101309172018981E5
:1057B0009A81820F931F0E94AC2A0E942D2A78940E
:1057C00081E0D2CF2F923F924F925F926F927F9261
:1057D0008F929F92AF92BF92CF92DF92EF92FF9201
:1057E0000F931F93CF93DF93CDB7DEB7CA1BDB0BAD
:1057F0000FB6F894DEBF0FBECDBF09942A88398852
:1058000048885F846E847D848C849B84AA84B98458
:10581000C884DF80EE80FD800C811B81AA81B98164
:10582000CE0FD11D0FB6F894DEBF0FBECDBFED0178
:105830000895AA1BBB1B51E107C0AA1FBB1FA617D7
:10584000B70710F0A61BB70B881F991F5A95A9F729
:1058500080959095BC01CD01089597FB072E16F415
:10586000009407D077FD09D00E94192C07FC05D0C1
:105870003EF4909581959F4F0895709561957F4F67
:105880000895EE0FFF1F0590F491E02D0994CF923B
:10589000DF92EF92FF92CF93DF93CDB7DEB72A97D7
:1058A0000FB6F894DEBF0FBECDBF89879A87A98552
:1058B000BA852D913D914D915C9129833A834B831B
:1058C0005C83232B242B252B41F424E239ED4BE57B
:1058D00057E029833A834B835C8369817A818B818A
:1058E0009C812DE133EF41E050E00E94272D6901BA
:1058F0007A01A7EAB1E49B01AC010E94462D6983BD
:105900007A838B839C83ACEEB4EFA70196010E944F
:10591000542D9B01AC0189819A81AB81BC81820F9E
:10592000931FA41FB51FB7FF03C00197A109B0487B
:10593000E985FA8580839183A283B3839F772A9632
:105940000FB6F894DEBF0FBECDBFDF91CF91FF90B1
:10595000EF90DF90CF9008950E94472C089580E04B
:1059600091E00E94472C0895B0E0A0E080930001F0
:1059700090930101A0930201B09303010895FB01EC
:10598000DC0104C08D910190801921F441505040F8
:10599000C8F7881B990B0895FB01DC0102C0019038
:1059A0000D9241505040D8F70895DC01CB01FC0125
:1059B000F999FECF06C0F2BDE1BDF89A319600B468
:1059C0000D9241505040B8F70895F999FECF92BD1D
:1059D00081BDF89A992780B50895A8E1B0E042E02A
:1059E00050E00C94D72CDC01A40FB51F415050405F
:1059F00048F0CB01840F951F2E910E94042D415039
:105A00005040D0F70895262FF999FECF92BD81BD61
:105A1000F89A019700B4021639F01FBA20BD0FB6EC
:105A2000F894FA9AF99A0FBE08950396272F0E94C8
:105A3000042D0E94032D252F0E94042D242F0C9449
:105A4000042D0196272F0E94042D0C94032D052E62
:105A500097FB1EF400940E943E2D57FD07D00E9434
:105A6000592D07FC03D04EF40C943E2D50954095D3
:105A7000309521953F4F4F4F5F4F089590958095FA
:105A8000709561957F4F8F4F9F4F08950E947B2D9A
:105A9000A59F900DB49F900DA49F800D911D112482
:105AA0000895B7FF0C94462D0E94462D821B930B40
:105AB0000895A1E21A2EAA1BBB1BFD010DC0AA1F4F
:105AC000BB1FEE1FFF1FA217B307E407F50720F067
:105AD000A21BB30BE40BF50B661F771F881F991FE2
:105AE0001A9469F760957095809590959B01AC012B
:105AF000BD01CF010895A29FB001B39FC001A39F34
:105B0000700D811D1124911DB29F700D811D1124F6
:105B1000911D0895F894FFCF23112F11591194115D
:105B2000CF110E124E1253125612711274127912B4
:105B30007C127F128212851288128B128E129112A1
:105B4000941299129C129F12D812111353135613C8
:105B50005913C913B6147615101671189918331AFB
:105B60009918331ACC18ED18331AEC19F9199F1B30
:105B7000A31B811B9B1BA71BAB1BAF1B141C7F1CF8
:105B80001C1CE61BEA1B201CEE1B241C301CFA1BF1
:105B9000781CFE1B341C021C381C601C061C3C1CA0
:105BA000671C0C1C421C4A1CF21B281CF61B2C1CDC
:105BB000101C461C561C701C761CE01B181C861CF6
:105BC0007C1D7C1DB41DB41D5D1E791EDC1DDC1DFD
:105BD0007E1E081F171F171F8F1C9D1CA41CA91CAD
:105BE000AE1CB31CB81CBD1CC21CC71CCC1CD11CD9
:105BF000D51CD71CD91C871B871B871B871B871BA2
:025C0000871B00
:105C0200010000000000000100000000000000048C
:105C12000100000004050000000000000909000066
:105C220000000000013204451031043E10371039E3
:105C320005FFFF0100FF000300FF82E200E900EA26
:105C420000B500B600B700CD008301CC008A0192F6
:105C52000194012102230224022502260227022A9C
:105C620002B300B4006F0070009F01CB019F02A03D
:105C720002D102946697C6F4F5F6F7313332003159
:105C820031295A1B750A1713120D0C05041614112B
:105C92000E0B0603FF15100F0A0702FFFFFFFF0995
:105CA20008012E2A2924231C1B2D2B2825221D1AEC
:105CB200FF2C2726211E19FFFFFFFF201F186E3F12
:105CC200662E6619660455025517552C623F4C3FE5
:105CD200442A441544003305331A332F2236222135
:105CE200220C110F112411390033001E783F802E2F
:105CF2008019800491029117912C843FA23FA22A1D
:105D0200A215A200B305B31AB32FC436C421C40C22
:105D1200D50FD524D539E633E61E00000000000079
:105D22000000000000000000000000000000000071
:105D32000000000000000000000000000000040459
:105D42000404040404040404040404040401040414
:105D52000404040404040404010401040404040407
:105D620004040404040108010808010800000000FA
:0E5D7200000000000000000000000000000023
:00000001FF
